:1000000009298030A100FE30A7200130A7207530DB
:10001000A7003030BE28A101A117AF00AF08031D13
:100020001328030114280130AF020310A20CA20C04
:10003000A20CC0302205403EAF07FE30A7202F089B
:10004000A728A101A117AF00FE30A7202F08A728DD
:10005000A401AA00AB01A01124080319A0150530C2
:10006000A3002730A900103041200330A900E83058
:100070004120A90164304120A9010A3041202A0809
:100080004828A8002B08A7002A08A600D220260886
:10009000A600A3030319A011240803195228230260
:1000A000031859282608031DA011A0195928303E0D
:1000B000A7280800AD0006118611831606118611C7
:1000C0000F30860583122D08A01884283E30A70023
:1000D0008030BE203330AC0098201330A700883029
:1000E000BE2098206430BD2098206430BD2022308E
:1000F000AC009820283083200C30832006308320E9
:10010000A0142D0884282014AC00201C92288611ED
:10011000033C031C972897200530A700DC30BE2045
:10012000031408002014FE3C0319A5288615201C82
:10013000201006150F3086052C08F03986040611AC
:10014000AC0E201898283230BD202D080429A11BA0
:100150005A2883178001840AFF3E031DAA28042918
:10016000A901A800FF30A807031CA907031C042944
:100170000330A700DF30BE20B228A701E83EA6006A
:10018000A709FC30031CC728A6070318C428A60724
:100190000000A70FC4282618CD28A61CD1280000CF
:1001A000D1280800AB01AA011030AC00270DAA0D20
:1001B000AB0D2808AA022908031C290FAB0203185B
:1001C000E8282808AA0729080318290FAB070310F5
:1001D000A60DA70DAC0BD628260804291030B000B8
:1001E000A701A601AD0CAC0C031CFC282808A6072F
:1001F00029080318290FA707A70CA60CAB0CAA0CFB
:10020000B00BF2282A080429831383120313000079
:100210000800A00107309F00E03083168500FF3002
:1002200086008113831285018601203084006030AE
:10023000AA20A03084005030AA2020308400303022
:10024000A920C830B020012077305A205A205A20E7
:100250002E305A2070305A2069305A2063305A208C
:1002600062305A2061305A2073305A2069305A2047
:1002700063305A202E305A206E305A206C305A206B
:100280000B30A900B830B120012044305A2043304F
:100290005A2046305A2031305A2036305A205530B4
:1002A0005A204B305A2042305A2020305A205A20AF
:1002B00056305A202D305A2032305A200730A900AB
:1002C000D030B120012041305A2064305A206A30A9
:1002D0005A2075305A2073305A2074305A202030FA
:1002E0005A204C305A2044305A2052305A20861816
:1002F0007F29851F7D2905147E2905107729012076
:1003000053305A2065305A2061305A2072305A20BA
:1003100063305A2068305A2020305A2073305A20D7
:1003200069305A2067305A206E305A2061305A2086
:100330006C305A20361405128316051283122A2AAD
:10034000C3013C03A500C90149082502031CB929C2
:10035000DC21B61CB7294308A6004908A200A60163
:10036000A20A0314A60DA20BB2292608C304C90FC2
:10037000A429B2014308B100B20CB10CB20CB10C0B
:10038000B20CB10CB20CB10C0F30B2053208AD009A
:100390003108AC00A9010A30A800EE20B1002B08FA
:1003A000B200B4014308B3000F30B3050030B40508
:1003B00031083307C3000800BA01B9010618F12952
:1003C0000130B020B90A0319BA0A0B303A02031CF3
:1003D000F029031DEF29B9303902031CF0294D2CF7
:1003E000DE299B30B0200618B614061CB610361C49
:1003F0000A2A440EB100B200F030B1050F30B20548
:100400003208A7003108A600A9013A30A800D2207E
:10041000BD001D2A8030A1000130A2003D080D2042
:100420000230A4004408292003013619013EB61801
:10043000013A03193611031D3615C40A851401301B
:10044000A900F430B1208510A901F030A8002808D7
:10045000B1200800BB01C4013612361ABF2ABA0106
:10046000B901061C442AB90A0319BA0A0130B0209E
:10047000AF303A02031C432A031D422AC930390215
:10048000031C432A4D2C312ABA01B9010618802ACF
:10049000B90A0319BA0A0A30B0203618742A390882
:1004A0000B3A3A04031D5F2A8030A1000130A200FC
:1004B0003D080D2035305A2039305A20732A39082A
:1004C000193A3A04031D662A8514732A39084B3AEF
:1004D0003A04031D6D2A8510732A3908FA3A3A0442
:1004E000031D732A4D2C7F2A11303A02031C7F2AE8
:1004F000031D7E2A95303902031C7F2A4D2C462A83
:1005000041303B02031C852A4D2CBB0A3A08031DCF
:100510008D2A65303902031C8E2A3616361CBE2AF7
:100520003B0EB100B200F030B1050F30B205320819
:10053000A7003108A600A9014130A800D220BD00C3
:100540008030A1008030212046305A206F305A2060
:1005500075305A206E305A2064305A2020305A208C
:1005600073305A2069305A2067305A206E305A2032
:1005700061305A206C305A2020305A202D2A361CE7
:10058000DB2A012049305A206E305A2069305A2027
:1005900074305A2069305A2061305A206C305A2009
:1005A00069305A207A305A2065305A202E305A202D
:1005B0005A205A20452B0830BD000130A2003D08CA
:1005C0000B20A101B61DF32A3B3041020318EA2A91
:1005D000C10AF22AC101173045020318F12AC50ADF
:1005E000F22AC501F72A4208C1004608C500051BCA
:1005F000072B4508031DFF2A0C30C700062B0D30C2
:100600004502031C062B0C304502C7000B2B450886
:10061000C70020305A200A3047020318112B20301F
:100620005A208030A100470828203A305A20023052
:10063000A400410829203A305A2030305A205A204C
:10064000051B2E2B0C3045020318292B61305A2034
:100650002B2B70305A200E30BD00302B0F30BD00D8
:10066000410803190130031D0301B5001E3041028A
:1006700003190130031D03013504B500013086184C
:10068000030135040319452B252C361E232CDC21B0
:100690000130C9000F3049020318512BDC21C90F6A
:1006A0004A2B3611B611DC21DC21DC21B61C5A2B79
:1006B00005145B2B05101230C900143049020318D1
:1006C000642BDC21C90F5D2BDC210730BC00A0218D
:1006D0004308C200DC21361D6E2BB6150630BC0067
:1006E000A0214308C600DC21361D772BB615063045
:1006F000BC00A0214308BE000330BC00A021430879
:10070000C8000530BC00A0214308C0000830BC0070
:10071000A0214308BF00DC21361D8F2BB615361CE7
:10072000952BB619942B36100120B619222C803047
:10073000A100803021203E08282020305A2001309E
:100740004002031DAA2B4A305A2061305A206E30D5
:100750005A20222C02304002031DB52B46305A206D
:1007600065305A2062305A20222C03304002031D8B
:10077000C02B4D305A2061305A2072305A20222C22
:1007800004304002031DCB2B41305A2070305A20D8
:1007900072305A20222C05304002031DD62B4D30DA
:1007A0005A2061305A2079305A20222C06304002DB
:1007B000031DE12B4A305A2075305A206E305A20E2
:1007C000222C07304002031DEC2B4A305A20753092
:1007D0005A206C305A20222C08304002031DF72B7F
:1007E00041305A2075305A2067305A20222C093067
:1007F0004002031D022C53305A2065305A207030BD
:100800005A20222C0A304002031D0D2C4F305A2052
:1008100063305A2074305A20222C0B304002031DC2
:10082000182C4E305A206F305A2076305A20222C05
:100830000C304002031D222C44305A2065305A20CF
:1008400063305A20242C4D2C2A2A851F2C2C05126B
:100850008316051283122E2C8316051683129B30E5
:10086000B020410803190130031D0301B500013018
:1008700086180301350403193E2C051585158514CA
:100880000130A900F430B120051185118510013027
:10089000A9004A30B120C40A482B01204E305A200A
:1008A0006F305A2020305A2073305A2069305A2035
:1008B00067305A206E305A2061305A206C305A20EE
:1008C000203084006030AA20A03084005030AA205C
:1008D000203084003030A9200618B616061CB61247
:1008E00003010618013EB61A013C031D7D2CB70A10
:1008F0000319B80A0130B020702C0301B61A013078
:10090000013A0319B612031DB61603010618013E7B
:10091000B61A013C031D922CB70A0319B80A01301C
:10092000B020852C03303802DE300319370203185B
:06093000602C36142A2A97
:02400E00503F21
:00000001FF
